:020000040000FA
:0400000005303A2865
:08000800A000030EA100831209
:1000100005191028831601178312B23081002B288E
:1000200083160113831203140B190310A80DA90DD5
:10003000AA0DAB0DAC0DAC16FF302C02031D2B2806
:10004000FA302B02031D2B2831152A08AF0029088E
:10005000AE002808AD008B100B11210E8300A00EFE
:04006000200E090065
:0C007400203084008001840A6030040207
:10008000031C3C281230B00096218316FF239000F9
:10009000831283160C308505870183128501870141
:1000A000073099000030831691009F008312C830FA
:1000B00083168100831231309000003083168C004B
:1000C000831210308B00831600309B001C141A081A
:1000D0008312BC00831610309B001C141A08831274
:1000E000BD00CD2181018E018F010B118B100B10F2
:1000F0008C018B17892031198C20B30B87280310B2
:1001000085190314B90DF030390203191121D521D5
:100110007A2864003210080031110130B7008B13C7
:100120002030370783169B001C141A088312A40082
:100130001030370783169B001C141A088312A30083
:10014000A6000230A6060030370783169B001C1459
:100150001A088312A200A7000130A7068B17321CD1
:10016000B72822090339A200A309A409A509240874
:100170002F02031D0B2923082E02031D0B29220821
:100180002D02031D0B2901303702031DCC283D1819
:10019000CC283D143E149D2102303702031DD52882
:1001A000BD18D528BD143E14A32103303702031D0A
:1001B000DE283D19DE283D153E14A9210430370202
:1001C000031DE728BD19E728BD153E14AF210530F2
:1001D0003702031DF0283D1AF0283D163E14B521C4
:1001E00006303702031DF928BD1AF928BD163E1442
:1001F000B62107303702031D02293D1B02293D1796
:100200003E14B72108303702031D0B29BD1B0B29F3
:10021000BD173E14B821B70A05303702031808008D
:100220008F280130B600B300B400B500B7008501D7
:100230008701B1138920B30B4929031085190314D1
:10024000B90DF030390203197029B40B4929013076
:1002500037020319B921023037020319BD210330D7
:1002600037020319C121043037020319C5210530B3
:1002700037020319C921063037020319CA21073092
:1002800037020319CB21083037020319CC219630ED
:10029000B400311D1A293111321C53292D0903399B
:1002A000AD00AE09AF092F1C1A298E018F010C1C5D
:1002B0001A290C102E1E1A298B1320303707BB0069
:1002C0002F08BA00832110303707BB002E08BA0070
:1002D000832100303707BB002D08BA0083218B171C
:1002E00085018701B70AB60105303702031C1A29B8
:1002F000CD2108003E1C08003E101030BB003D0818
:10030000BA00832108008B133A0883161C159A0043
:100310003B089B0055309D00AA309D009C14640052
:100320009C188F291C1183128B170800FF30D000F6
:10033000D415D515D615D71508000F30D204BD1029
:100340003D11BD1108000F30D2043D103D11BD110B
:1003500008000F30D2043D10BD10BD1108000F3051
:10036000D2043D10BD103D1108000800080008002F
:1003700008000508023A850008000508013A8500D2
:1003800008000508203A850008000508103A850095
:10039000080008000800080008003D08D200031DFE
:1003A00008001130BD00D20008008F0803190800B2
:1003B0008F01D00F632AD00A0E305205031DEF299A
:1003C000541DE529D4015416FD29D41DEA29D40170
:1003D0005416FD29541EFD29D401D414FD29D41C22
:1003E000F429D4015415FD29541DF929D401D4153B
:1003F000FD29541EFD29D40154150D305205031D4D
:10040000102A551D062AD50155161E2AD51D0B2A60
:10041000D50155161E2A551E1E2AD501D5141E2A91
:10042000D51C152AD50155151E2A551D1A2AD50188
:10043000D5151E2A551E1E2AD50155150B305205FD
:10044000031D312A561D272AD60156163F2AD61DCE
:100450002C2AD60156163F2A561E3F2AD601D614FC
:100460003F2AD61C362AD60156153F2A561D3B2A4E
:10047000D601D6153F2A561E3F2AD60156150730FB
:100480005205031D522A571D482AD7015716602AC4
:10049000D71D4D2AD7015716602A571E602AD7014B
:1004A000D714602AD71C572AD7015715602A571D21
:1004B0005C2AD701D715602A571E602AD701571525
:1004C0007A213D08D2005008D1000C305405031D9C
:1004D00085100C305505031D05100C305605031D05
:1004E00085120C305705031D051251080E02031822
:1004F0008D2A12305405031D851412305505031D35
:10050000051412305605031D851612305705031DBC
:100510000516FF305002031908008F08031D08005C
:10052000892051080E02031C8D2A18305405031D22
:10053000851006305405031D851418305505031D1C
:10054000051006305505031D051418305605031D0A
:10055000851206305605031D851618305705031DF4
:0C056000051206305705031D05160800A3
:084000000400030003000800A6
:02400E00CC01E3
:10420000010078007A007C007E007B0079007F004E
:104210007D007A0078007E007C00FF00FF00FF0038
:104220000000F200F600FA00FE00F200F600FA00CC
:10423000FE00F200F600FA00FE00FF00FF00FF00A3
:10424000010005000500050005000900090009003E
:1042500009000D000D000D000D00FF00FF00FF0024
:10426000FF00FF00FF00FF00FF00FF00FF00FF0056
:10427000FF00FF00FF00FF00FF00FF00FF00FF0046
:10428000FF00FF00FF00FF00FF00FF00FF00FF0036
:10429000FF00FF00FF00FF00FF00FF00FF00FF0026
:1042A000FF00FF00FF00FF00FF00FF00FF00FF0016
:1042B000FF00FF00FF00FF00FF00FF00FF00FF0006
:1042C000FF00FF00FF00FF00FF00FF00FF00FF00F6
:1042D000FF00FF00FF00FF00FF00FF00FF00FF00E6
:1042E000FF00FF00FF00FF00FF00FF00FF00FF00D6
:1042F000FF00FF00FF00FF00FF00FF00FF00DD00E8
:00000001FF
